:100000000C943D010C9465010C9465010C94650100
:100010000C9465010C9465010C9465010C946501C8
:100020000C9465010C9465010C94D4040C94F805AF
:100030000C9465010C9465010C9465010C946501A8
:100040000C9465010C9465010C9465010C94650198
:100050000C9465010C9465010C9465010C940502E7
:100060000C9465010C9465010C9465010C94650178
:100070000C9465010C9465010C9465010C94650168
:100080000C9465010C9465010C9465010C94650158
:100090000C9465010C9465010C9465010C94650148
:1000A0000C9465010C9465010C94650105A84CCD78
:1000B000B2D44EB93836A9020C50B9918688083CA2
:1000C000A6AAAA2ABE000000803F05010902A101DC
:1000D0000901A10085010509190129031500250160
:1000E00095037501810295017505810305010930AC
:1000F000093109381581257F750895038106C0C02F
:1001000005010906A1018502050719E029E7150087
:1001100025017501950881029501750881039506F1
:100120007508150025650507190029658100C009B6
:100130000402000103000000092101010001226501
:1001400000070584034000010000000000000000DB
:100150002A2B280000000000000000000000000022
:1001600000000000000000002C9EB4A0A1A2A43456
:10017000A6A7A5AE362D3738271E1F2021222324FF
:100180002526B333B62EB7B89F8485868788898A9B
:100190008B8C8D8E8F909192939495969798999A37
:1001A0009B9C9D2F3130A3AD350405060708090A35
:1001B0000B0C0D0E0F101112131415161718191A17
:1001C0001B1C1DAFB1B0B50004030904220341009C
:1001D00072006400750069006E006F0020004C0022
:1001E00065006F006E006100720064006F0018030C
:1001F000410072006400750069006E006F0020000D
:100200004C004C004300120100020000004041235A
:10021000340000010102000112010002020000404E
:100220004123340000010102000100C18081C108A6
:100230000B0002020201000904000001020200009A
:1002400005240010010524010101042402060524EF
:100250000600010705810310004009040100020A9D
:10026000000000070502024000000705830240006D
:1002700000006801150339055A0711241FBECFEF8E
:10028000DAE0DEBFCDBF11E0A0E0B1E0E2E7F5E1EA
:1002900002C005900D92AA32B107D9F711E0AAE287
:1002A000B1E001C01D92A535B107E1F712E0CAE740
:1002B000D2E004C02297FE010E94B30AC237D107E0
:1002C000C9F70E94DB030C94B70A0C940000089550
:1002D000809102019091030190932D0180932C0154
:1002E00008955F926F927F928F929F92AF92BF928A
:1002F000CF92DF92EF92FF920F931F93E090000155
:10030000F090010180912A0190912B010196B70193
:100310000E948A0A9C0190932B0180932A01442712
:1003200037FD4095542FCA01B9010E940D0928EDEF
:100330003FE049EC50E40E94DB095B016C010027BF
:10034000F7FC0095102FC801B7010E940D099B0111
:10035000AC01C601B5010E9472087B018C0160915D
:10036000020170910301882777FD8095982F0E94E4
:100370000D093B014C01B701C8010E946F089B01A8
:10038000AC01C401B3010E94DB090E94DA085B01E1
:100390006C01562EB701C8010E943E0A9B01AC01B8
:1003A000C401B3010E94DB090E94DA087B018C01C1
:1003B00080912C01581A80912E014E2D481B89E303
:1003C00091E0652D20E00E94AC03A0922C01B09238
:1003D0002D01E0922E01F0922F01609104017091A5
:1003E0000501882777FD8095982F0E944D021F9167
:1003F0000F91FF90EF90DF90CF90BF90AF909F90C4
:100400008F907F906F905F9008951F920F920FB61C
:100410000F9211242F933F938F939F93AF93BF938A
:100420008091340190913501A0913601B09137014E
:10043000309138010196A11DB11D232F2D5F2D375D
:1004400020F02D570196A11DB11D209338018093F6
:10045000340190933501A0933601B0933701809118
:10046000300190913101A0913201B0913301019698
:10047000A11DB11D8093300190933101A0933201F1
:10048000B0933301BF91AF919F918F913F912F9185
:100490000F900FBE0F901F9018959B01AC017FB776
:1004A000F8948091300190913101A0913201B09186
:1004B000330166B5A89B05C06F3F19F00196A11DD9
:1004C000B11D7FBFBA2FA92F982F8827860F911DA6
:1004D000A11DB11D62E0880F991FAA1FBB1F6A955D
:1004E000D1F7BC012DC0FFB7F894809130019091F5
:1004F0003101A0913201B0913301E6B5A89B05C04E
:10050000EF3F19F00196A11DB11DFFBFBA2FA92F12
:10051000982F88278E0F911DA11DB11DE2E0880F35
:10052000991FAA1FBB1FEA95D1F7861B970B885E00
:100530009340C8F2215030404040504068517C4FB9
:10054000211531054105510571F60895789484B55A
:10055000826084BD84B5816084BD85B5826085BDBF
:1005600085B5816085BDEEE6F0E0808181608083A5
:10057000E1E8F0E010828081826080838081816088
:100580008083E0E8F0E0808181608083E1EBF0E04F
:10059000808184608083E0EBF0E0808181608083F3
:1005A000E1E9F0E0808182608083808181608083E6
:1005B000E0E9F0E0808181608083E1ECF0E080811F
:1005C00082608083808181608083E0ECF0E08081C4
:1005D00081608083EAE7F0E08081846080838081AD
:1005E0008260808380818160808380818068808355
:1005F0000895FC0191818081813A31F4913089F034
:1006000080E0933089F40DC0813269F49B3021F48D
:1006100082818093060105C09A3029F482818093FB
:10062000070181E0089580E0089510923901109249
:100630003D0110923C0186E191E090933B01809353
:100640003A0110923F0110923E010895EF92FF92FD
:100650000F931F93DF93CF930F92CDB7DEB78983AC
:100660008B017A0184E0BE016F5F7F4F41E050E073
:100670000E943A0584E4B801A7010E943A050F9050
:10068000CF91DF911F910F91FF90EF90089582E03D
:1006900048E050E00E9426030895EF92FF920F93E6
:1006A0001F93DF93CF93CDB7DEB728970FB6F8949B
:1006B000DEBF0FBECDBF7C019E012F5F3F4F88E0A4
:1006C000F90111928A95E9F7F701A481B581109794
:1006D00059F0ED91FC9111970190F081E02DCD0141
:1006E00070E0A901099518C067FD07C0E62FF0E08A
:1006F000E85BFE4F6491662341F481E090E0F701EE
:100700009383828320E030E019C067FF04C08981B1
:10071000826089836F776B83C7018E010F5F1F4FE4
:10072000B8010E94470388E0F80111928A95E9F721
:10073000C701B8010E94470321E030E0C9012896B3
:100740000FB6F894DEBF0FBECDBFCF91DF911F91E2
:100750000F91FF90EF900895DF93CF9300D000D0DA
:10076000CDB7DEB7FC01808189836A834B832C83FC
:1007700081E0BE016F5F7F4F44E050E00E9426039E
:100780000F900F900F900F90CF91DF91089580E818
:100790006AEC70E045E650E00E946E040895FC01AA
:1007A00080818F5F808380E86FE271E049E150E0F3
:1007B0000E946E040895CF93DF930E94A60288E4FE
:1007C00091E00E9420050E946701C0E0D0E00E94F5
:1007D00071012097E1F30E940000F9CFCF92DF92E0
:1007E000EF92FF920F931F93CF93DF937C016B01E6
:1007F0008A01C0E0D0E00FC0D6016D916D01D70134
:10080000ED91FC910190F081E02DC7010995C80F91
:10081000D91F015010400115110571F7CE01DF916C
:10082000CF911F910F91FF90EF90DF90CF9008959F
:100830009FB7F89487708093E9008091F2009FBF82
:100840000895282F809142018823C1F057FF1AC0D4
:1008500015C02898909341018091F1008193E2178F
:10086000F307B9F74115510539F08091F20088235B
:1008700019F48BE68093E800AFBF02C04FEF5FEF43
:10088000CA010895AFB7F89427702093E9008091CA
:10089000F200282F30E0241735070CF4A901FB01E2
:1008A0009B01240F311D94E6DACFDF93CF930F9293
:1008B000CDB7DEB7BE016F5F7F4F41E050E00E94D1
:1008C0002104019719F02FEF3FEF03C08981282FF2
:1008D00030E0C9010F90CF91DF910895FF920F93FF
:1008E0001F93F82E142F052F40914501509146017A
:1008F000212F302FC901DC01FB016EEF29C0F7FE6B
:1009000002C0949101C09081209143013091440133
:1009100024173507ACF48091E8008570E1F38091ED
:10092000E80082FF03C02FEF3FEF17C09093F10064
:10093000C90101968F739070892B11F46093E800C0
:100940002F5F3F4F3093440120934301119731961D
:100950001097A9F6812F902F9C01C9011F910F912B
:10096000FF9008959C018091E80082FFFCCFF9017F
:10097000260F311D03C08091F1008193E217F30728
:10098000D1F7289884E6809341018BEF8093E800AB
:10099000CB0108958093E9008091F200882319F03B
:1009A0008AE38093E80008951F920F920FB60F928A
:1009B00011248F939F938091E1001092E100982F72
:1009C00083FF0FC01092E90081E08093EB0010924A
:1009D000EC0082E38093ED001092420188E0809366
:1009E000F00092FF26C083E08093E9008091F2003E
:1009F000882319F08AE38093E800809140018823DE
:100A000051F08091400181508093400180914001DC
:100A1000882309F45D9A80914101882351F08091E7
:100A2000410181508093410180914101882309F463
:100A3000289A9F918F910F900FBE0F901F9018953D
:100A40001092420181E08093D70080EA8093D80021
:100A500082E189BD09B400FEFDCF80E98093D80012
:100A60008CE08093E2001092E000559A209A08955D
:100A7000089508955F926F927F928F929F92AF92A6
:100A8000BF92CF92DF92EF92FF920F931F93CF937B
:100A9000DF93E82E842E752E80914201882371F118
:100AA0008B01242F352FC901EC017AEFF72E67E077
:100AB000962E9E2050E4552E8E2D90E040E2A42EDE
:100AC000B12CA822B9223AE3632E20E4C22ED12C05
:100AD000C822D92258C09FB7F8949092E90080911B
:100AE000E80085FD02C020E004C08091F200252DC1
:100AF000281B9FBF222361F4FA9419F42FEF3FEFD4
:100B00004DC061E070E080E090E00E944D023BC08B
:100B1000822F90E0C817D9070CF42C2FC21BD109E3
:100B20004FB7F8949092E900A114B10421F406C0E3
:100B30001092F10021502223D9F719C0E7FC03C01D
:100B4000F801922F10C0C801322F06C0FC01019697
:100B5000E491E093F10031503323C1F706C0819155
:100B60008093F10091509923D1F7020F111D8091CC
:100B7000E80085FF05C0209729F4C114D10411F0C5
:100B80006092E8004FBF209709F0A5CF5D9884E6FA
:100B900080934001282D372DC9019C01C901DF91A7
:100BA000CF911F910F91FF90EF90DF90CF90BF906A
:100BB000AF909F908F907F906F905F9008950F936C
:100BC0001F93DF93CF930F92CDB7DEB719828E01BB
:100BD0000F5F1F4FC8010E94C107C8010E94CF03C9
:100BE000898190E00F90CF91DF911F910F9108952F
:100BF0001F920F920FB60F921124EF92FF921F9344
:100C00002F933F934F935F936F937F938F939F9314
:100C1000AF93BF93EF93FF93DF93CF93CDB7DEB73F
:100C20006197DEBFCDBF1092E9008091E80083FF9D
:100C30000FC1FE0131969E01275F3F4F03C0809197
:100C4000F1008193E217F307D1F7289884E68093A7
:100C5000410182EF8093E800998197FF05C0809160
:100C6000E80080FFFCCF03C08EEF8093E800292FBF
:100C700030E0C90180769070892B09F0C2C08A816A
:100C8000882329F41092F1001092F100D6C081302F
:100C900009F4D3C0833009F4D0C0853049F4809181
:100CA000E80080FFFCCF8B8180688093E300C5C0A3
:100CB000863009F07CC01C81EF80F8841230C1F5C9
:100CC0001092E900109244011092430110924601E3
:100CD000109245010E94DF0599E0FE013996DF017F
:100CE000292F1D922A95E9F799871A8791E09E8707
:100CF00090E8988B9AEF998B2091430130914401B1
:100D0000275F3F4F3C872B878D871092E900109219
:100D1000440110924301F0924601E092450180E0C7
:100D2000BF0149E050E00E946E040E94DF0585C0CB
:100D30001092E9001092440110924301F092460192
:100D4000E0924501123241F482E290E00E94C70332
:100D5000892B09F476C071C0113079F488E0E81667
:100D6000F10419F481E080934701809147018823C1
:100D700009F06BC0E6E0F2E013C0133009F061C087
:100D80008B81882319F4E8ECF1E00AC0823019F471
:100D9000ECECF1E005C0813009F053C0EEEEF1E07B
:100DA000449180E8BF0150E00E946E0446C0873045
:100DB00009F447C0883021F481E08093F1003DC000
:100DC0008930D9F523703070232BD9F5EBE2F2E0AE
:100DD00091E031E026E39093E9003093EB008491B9
:100DE0008093EC002093ED009F5F3196953099F74A
:100DF0008EE78093EA001092EA008B818093420193
:100E00001CC08F8198851092E900109244011092C5
:100E1000430190934601809345018D81882329F4F5
:100E2000CE0101960E94D50706C0823051F4CE0152
:100E300001960E94F902882321F08EEF8093E8004A
:100E400007C081E28093EB0003C0E8E1F2E0A8CFA5
:100E50006196DEBFCDBFCF91DF91FF91EF91BF9142
:100E6000AF919F918F917F916F915F914F913F9142
:100E70002F911F91FF90EF900F900FBE0F901F903A
:100E80001895DC0180910801909109018F5F9F4FB7
:100E900061F4ED91FC9111970680F781E02DCD0171
:100EA0000995909309018093080180910801909120
:100EB0000901089510924C0110924B0188EE93E0C5
:100EC000A0E0B0E080934D0190934E01A0934F01BC
:100ED000B09350018EE191E090934A0180934901D3
:100EE00008950F931F93DF93CF930F92CDB7DEB783
:100EF0008C01698380911101882369F083E0BE0130
:100F00006F5F7F4F41E050E00E943A0518161906C6
:100F100014F49C0107C081E090E0F8019383828380
:100F200020E030E0C9010F90CF91DF911F910F9128
:100F3000089583E00E94CA04089520910801309129
:100F400009018FEF2F3F380739F08FEF9FEF909314
:100F500009018093080104C082E00E9455049C01AD
:100F6000C901089582E00E941804282F8091080189
:100F7000909109018F5F9F4F09F02F5F822F90E0C2
:100F80000895FC0180818E5F808380E86FE272E0CB
:100F900042E450E00E946E04089588E491E00E94CB
:100FA0003805F8940C94003C0895CF93DF93EC013E
:100FB00089819881913A51F4813269F580E06AE043
:100FC00071E047E050E00E946E0423C0913219F5B1
:100FD000803239F48AE091E067E070E00E94B20468
:100FE00018C08232C1F480911101882379F0809178
:100FF0000A0190910B01A0910C01B0910D01805B51
:101000009440A040B04011F40E94CD078A818093A3
:10101000110181E001C080E0DF91CF91089541D1BD
:1010200030F046D120F031F49F3F11F41EF436C168
:101030000EF4E095E7FB2CC1E92F94D180F3BA17A9
:10104000620773078407950718F071F49EF5ACC129
:101050000EF4E0950B2EBA2FA02D0B01B9019001D3
:101060000C01CA01A0011124FF27591B99F0593F17
:1010700050F4503E68F11A16F040A22F232F342F5F
:101080004427585FF3CF469537952795A795F040AD
:101090005395C9F77EF41F16BA0B620B730B840BC2
:1010A000BAF09150A1F0FF0FBB1F661F771F881F7A
:1010B000C2F70EC0BA0F621F731F841F48F48795D2
:1010C00077956795B795F7959E3F08F0B3CF9395C1
:1010D000880F08F09927EE0F979587950895F0D01F
:1010E000E3952FC10CD01CC1E3D040F0DAD030F032
:1010F00021F45F3F19F0CCC0511157C1CFC032D19C
:1011000098F39923C9F35523B1F3951B550BBB27CE
:10111000AA2762177307840738F09F5F5F4F220F7B
:10112000331F441FAA1FA9F333D00E2E3AF0E0E874
:1011300030D091505040E695001CCAF729D0FE2FC0
:1011400027D0660F771F881FBB1F26173707480752
:10115000AB07B0E809F0BB0B802DBF01FF27935808
:101160005F4F2AF09E3F510568F092C01EC15F3F5D
:10117000ECF3983EDCF3869577956795B795F795F0
:101180009F5FC9F7880F911D9695879597F90895E8
:10119000E1E0660F771F881FBB1F62177307840784
:1011A000BA0720F0621B730B840BBA0BEE1F88F793
:1011B000E095089504D06894B111F7C00895DAD08D
:1011C00088F09F5790F0B92F9927B751A0F0D1F030
:1011D000660F771F881F991F1AF0BA95C9F712C0BA
:1011E000B13081F0E1D0B1E00895DEC0672F782FF3
:1011F0008827B85F39F0B93FCCF386957795679526
:10120000B395D9F73EF490958095709561957F4F91
:101210008F4F9F4F0895E89409C097FB3EF4909537
:101220008095709561957F4F8F4F9F4F9923A9F0BF
:10123000F92F96E9BB279395F6958795779567954E
:10124000B795F111F8CFFAF4BB0F11F460FF1BC092
:101250006F5F7F4F8F4F9F4F16C0882311F096E925
:1012600011C0772321F09EE8872F762F05C06623D3
:1012700071F096E8862F70E060E02AF09A95660F8C
:10128000771F881FDAF7880F9695879597F9089545
:1012900097F99F6780E870E060E008959FEF80EC29
:1012A000089500240A9416161706180609060895CC
:1012B00000240A9412161306140605060895EECFAC
:1012C00059D0E8F3E894EFEFBB273FE048EC5FE745
:1012D0006B3D73078407950708F1FF279F57B25AA4
:1012E0006A4D7F40894CF04032F4BE556542704FE4
:1012F0008643FF4F0894EE1F915030F0BB0F661FDE
:10130000771F881FFF1FEBCF9EE7882332F0BB0FAC
:10131000661F771F881F9A95C1F79395E095B4C013
:10132000092E0394000C11F4882352F0BB0F40F4F3
:10133000BF2B11F460FF04C06F5F7F4F8F4F9F4F33
:101340000895EF93E0FF06C0A2EA2AED3FE049ECE2
:101350005FEB72DEE5DF0F90039401FC9058ECEA3E
:10136000F0E0A2C057FD9058440F551F59F05F3F61
:1013700071F04795880F97FB991F61F09F3F79F0B7
:1013800087950895121613061406551FF2CF469539
:10139000F1DF08C0161617061806991FF1CF8695BB
:1013A0007105610508940895E894BB27662777279F
:1013B000CB0197F908950BD0B3CF73DF28F078DF16
:1013C00018F0952309F064CF69CF1124EECFCADF5E
:1013D000A0F3959FD1F3950F50E0551F629FF00148
:1013E000729FBB27F00DB11D639FAA27F00DB11DA1
:1013F000AA1F649F6627B00DA11D661F829F22272A
:10140000B00DA11D621F739FB00DA11D621F839FB0
:10141000A00D611D221F749F3327A00D611D231F86
:10142000849F600D211D822F762F6A2F11249F57D4
:1014300050408AF0E1F088234AF0EE0FFF1FBB1FF7
:10144000661F771F881F91505040A9F79E3F510596
:1014500070F01ECFAACF5F3FECF3983EDCF3869589
:1014600077956795B795F795E7959F5FC1F7FE2B41
:10147000880F911D9695879597F908959F9320DF82
:101480000F9007FCEE5F5DCF9F3F49F0915028F42D
:10149000869577956795B7959F5F80389F4F880FA2
:1014A0009695879597F908959F938F937F936F9360
:1014B000FF93EF939B01AC017EDFEF91FF9105D08D
:1014C0002F913F914F915F9176CFDF93CF931F93F1
:1014D0000F93FF92EF92DF927B018C01689405C01D
:1014E000DA2EEF0174DFFE01E894A5912591359184
:1014F00045915591AEF3EF019FDDFE019701A801E3
:10150000DA9479F7DF90EF90FF900F911F91CF91D0
:10151000DF91089597FB092E07260AD077FD04D0A6
:101520000CD006D000201AF4709561957F4F089575
:10153000F6F7909581959F4F0895AA1BBB1B51E12B
:1015400007C0AA1FBB1FA617B70710F0A61BB70B33
:10155000881F991F5A95A9F780959095BC01CD01D8
:101560000895EE0FFF1F0590F491E02D0994F89473
:02157000FFCFAB
:101572006400640002000101FFFF00E100000000BE
:101582000000000000004D03EE03000000007107A0
:0A159200EE03B2079D074107990719
:00000001FF
